** EXPERIMENTAL (HLL) ** Open Watcom Linker Version 1.6beta1 Limited Availability
Portions Copyright (c) 1985-2002 Sybase, Inc. All Rights Reserved.
Created on:       12/01/07 18:55:31
Warning! W1121: file U:/tmp\ldconv_gdbmmodule_obj_dbef4f08017a1c96a8.obj(U:\DEV\python-2.7.2\Modules\gdbmmodule.c): '_initgdbm' has already been exported
Executable Image: build/lib.os2knix-2.7/gdbm.pyd
creating an OS/2 EMX dynamic link library


                        +------------+
                        |   Groups   |
                        +------------+

Group                           Address              Size
=====                           =======              ====

CGROUP                          0001:00000000        00004e40
DGROUP                          0002:00000000        00000f60



                        +--------------+
                        |   Segments   |
                        +--------------+

Segment                Class          Group          Address         Size
=======                =====          =====          =======         ====

TEXT32                 CODE           CGROUP         0001:00000000   00004e40
________TEXT           CODE           CGROUP         0001:00004e40   00000000
DATA32                 DATA           DGROUP         0002:00000000   00000ed0
SET1__os2dll           DATA           DGROUP         0002:00000ed0   00000004
SET2__os2dll           DATA           DGROUP         0002:00000ed4   00000000
SET3__os2dll           DATA           DGROUP         0002:00000ed4   00000004
SET1___CTOR_LIST__     DATA           DGROUP         0002:00000ed8   00000004
SET2___CTOR_LIST__     DATA           DGROUP         0002:00000edc   00000000
SET3___CTOR_LIST__     DATA           DGROUP         0002:00000edc   00000004
SET1___DTOR_LIST__     DATA           DGROUP         0002:00000ee0   00000004
SET2___DTOR_LIST__     DATA           DGROUP         0002:00000ee4   00000000
SET3___DTOR_LIST__     DATA           DGROUP         0002:00000ee4   00000004
SET1___crtinit1__      DATA           DGROUP         0002:00000ee8   00000004
SET2___crtinit1__      DATA           DGROUP         0002:00000eec   00000000
SET3___crtinit1__      DATA           DGROUP         0002:00000eec   00000004
SET1___crtexit1__      DATA           DGROUP         0002:00000ef0   00000004
SET2___crtexit1__      DATA           DGROUP         0002:00000ef4   00000000
SET3___crtexit1__      DATA           DGROUP         0002:00000ef4   00000004
SET1___eh_frame__      DATA           DGROUP         0002:00000ef8   00000004
SET2___eh_frame__      DATA           DGROUP         0002:00000efc   00000000
SET3___eh_frame__      DATA           DGROUP         0002:00000efc   00000004
SET1___eh_init__       DATA           DGROUP         0002:00000f00   00000004
SET2___eh_init__       DATA           DGROUP         0002:00000f04   00000000
SET3___eh_init__       DATA           DGROUP         0002:00000f04   00000004
SET1___eh_term__       DATA           DGROUP         0002:00000f08   00000004
SET2___eh_term__       DATA           DGROUP         0002:00000f0c   00000000
SET3___eh_term__       DATA           DGROUP         0002:00000f0c   00000004
SET1___fork_parent1__  DATA           DGROUP         0002:00000f10   00000004
SET2___fork_parent1__  DATA           DGROUP         0002:00000f14   00000000
SET3___fork_parent1__  DATA           DGROUP         0002:00000f14   00000004
SET1___fork_child1__   DATA           DGROUP         0002:00000f18   00000004
SET2___fork_child1__   DATA           DGROUP         0002:00000f1c   00000000
SET3___fork_child1__   DATA           DGROUP         0002:00000f1c   00000004
________DATA           DATA           DGROUP         0002:00000f20   00000000
BSS32                  BSS            DGROUP         0002:00000f20   00000040
c_common               BSS            DGROUP         0002:00000f60   00000000
________BSS            BSS            DGROUP         0002:00000f60   00000000


                        +----------------+
                        |   Memory Map   |
                        +----------------+

* = unreferenced symbol
+ = symbol only referenced locally

Address        Symbol
=======        ======

Module: U:\usr\lib\dll0hi.obj({standard input})
0001:00000000* __text
0002:00000000* __data
0002:00000000* ___data_start
0002:00000f20* ___bss_start
0002:00000ed0+ __os2dll
0002:00000ed8  ___CTOR_LIST__
0002:00000ee0  ___DTOR_LIST__
0002:00000ee8* ___crtinit1__
0002:00000ef0* ___crtexit1__
0002:00000ef8* ___eh_frame__
0002:00000f00  ___eh_init__
0002:00000f08  ___eh_term__
0002:00000f10+ ___fork_parent1__
0002:00000f18+ ___fork_child1__
Module: U:/tmp\ldconv_gdbmmodule_obj_dbef4f08017a1c96a8.obj(U:\DEV\python-2.7.2\Modules\gdbmmodule.c)
0001:000000c1  _initgdbm
Module: U:\usr\local446\lib\libc_dll.lib(dllinit.obj)
0001:00000c60  _DLL_InitTerm
Module: U:\usr\lib\libend.lib(src/libend/386/endlink386.asm)
0002:00000f60  _end
0002:00000f20  _edata
Module: U:\usr\lib\libend.lib(src/libend/386/end.asm)
0001:00004e40* _etext
0001:00004e40* __etext
0000:00000000  WEAK$ZERO
0002:00000f60  __end
0002:00000f20  __edata
Module: U:\extras\lib\gdbm.lib(gdbmstore.obj)
0001:00000cd8  _gdbm_store
Module: U:\extras\lib\gdbm.lib(gdbmdelete.obj)
0001:00001070  _gdbm_delete
Module: U:\extras\lib\gdbm.lib(global.obj)
0002:00000f30* __gdbm_file
0002:00000f34* __gdbm_memory
0002:00000f3c* __gdbm_fetch_val
0002:00000f40  _gdbm_errno
Module: U:\extras\lib\gdbm.lib(gdbmerrno.obj)
0001:00001480* _gdbm_errlist
0001:000014e2  _gdbm_strerror
Module: U:\extras\lib\gdbm.lib(gdbmfetch.obj)
0001:0000152d  _gdbm_fetch
Module: U:\extras\lib\gdbm.lib(gdbmexists.obj)
0001:00001610  _gdbm_exists
Module: U:\extras\lib\gdbm.lib(gdbmseq.obj)
0001:000017e2  _gdbm_firstkey
0001:00001825  _gdbm_nextkey
Module: U:\extras\lib\gdbm.lib(gdbmopen.obj)
0001:000018c0  _gdbm_open
0001:00002360  __gdbm_init_cache
Module: U:\extras\lib\gdbm.lib(gdbmsync.obj)
0001:00002500  _gdbm_sync
Module: U:\extras\lib\gdbm.lib(gdbmreorg.obj)
0001:00002530  _gdbm_reorganize
Module: U:\extras\lib\gdbm.lib(gdbmclose.obj)
0001:00002a40  _gdbm_close
Module: U:\tmp\ldconv_gcc_a_dbef4f08017a1d6d80.lib(emx-ctordtor.obj)
0001:00002ba0  ___ctordtorInit
0001:00002bac* ___POST$__ctordtorInit
0001:00002bdc  ___ctordtorTerm
0001:00002be9* ___POST$__ctordtorTerm
Module: U:\extras\lib\gdbm.lib(findkey.obj)
0001:00002c45  __gdbm_read_entry
0001:00002e4a  __gdbm_findkey
Module: U:\extras\lib\gdbm.lib(falloc.obj)
0001:000030c0  __gdbm_alloc
0001:000031a6  __gdbm_free
0001:00003937  __gdbm_put_av_elem
Module: U:\extras\lib\gdbm.lib(bucket.obj)
0001:00003d00  __gdbm_new_bucket
0001:00003db7  __gdbm_get_bucket
0001:00004a12  __gdbm_write_bucket
0001:00004097  __gdbm_split_bucket
Module: U:\extras\lib\gdbm.lib(update.obj)
0001:00004d25  __gdbm_fatal
0001:00004b85  __gdbm_end_update
Module: U:\extras\lib\gdbm.lib(hash.obj)
0001:00004db0  __gdbm_hash


                        +----------------------+
                        |   Imported Symbols   |
                        +----------------------+

Symbol                              Module
======                              ======

___libc_ForkRegisterModule          libc064
___init_dll                         libc064
___libc_Back_termDll                libc064
___libc_ForkDeregisterModule        libc064
__atfork_callback                   libc064
_PyType_Type                        python27
_Py_InitModule4                     python27
_PyModule_GetDict                   python27
_PyErr_NewException                 python27
_PyDict_SetItemString               python27
_PyString_FromString                python27
_PyArg_Parse                        python27
__errno                             libc064
_PyErr_SetFromErrno                 python27
_PyExc_KeyError                     python27
_PyErr_SetString                    python27
_PyExc_TypeError                    python27
_PyString_FromStringAndSize         python27
_PyErr_Format                       python27
__Py_NoneStruct                     python27
_PyArg_ParseTuple                   python27
_PyOS_snprintf                      python27
__PyObject_New                      python27
_Py_FindMethod                      python27
_PyInt_FromLong                     python27
_PyList_New                         python27
_PyList_Append                      python27
__PyErr_BadInternalCall             python27
_PyObject_Free                      python27
__CRT_init                          libc064
__CRT_term                          libc064
__std_free                          libc064
___ctordtorInit1                    libc064
___ctordtorTerm1                    libc064
__std_bcopy                         libc064
__std_lseek                         libc064
__std_write                         libc064
__std_malloc                        libc064
__std_strlen                        libc064
__std_strcpy                        libc064
__std_open                          libc064
__std_fstat                         libc064
__std_close                         libc064
__std_flock                         libc064
__std_ftruncate                     libc064
__std_fsync                         libc064
__std_read                          libc064
__std_unlink                        libc064
__std_rename                        libc064
__std_bcmp                          libc064
__std_printf                        libc064
__std_exit                          libc064


                        +--------------------+
                        |   Libraries Used   |
                        +--------------------+

U:\extras\lib\gdbm.lib
U:\tmp\ldconv_python2_7_dll_a_dbef4f08017a1d2730.lib
U:\tmp\ldconv_gcc_a_dbef4f08017a1d6d80.lib
U:\usr\lib\libc_alias.lib
U:\usr\local446\lib\libc_dll.lib
U:\usr\lib\libend.lib


                        +-----------------------+
                        |   Linker Statistics   |
                        +-----------------------+

Stack size:  0000 (0.)
Memory size:  5da0 (23968.)
Link time: 00:00.09
